:020000040800F2
:1000000018070020D10000086D1500080113000832
:1000100000000000000000000000000000000000E0
:10002000000000000000000000000000B51F0008F4
:100030000000000000000000111700080122000865
:100040000101000801010008010100080101000888
:1000500001010008E10D000801010008010100088C
:1000600001010008010100083D0C00080101000821
:100070000101000801010008010100080101000858
:100080000101000895220008010100080101000893
:100090000101000801010008010100080101000838
:1000A0000101000801010008010100083D240008C9
:1000B00079240008A12400080101000803488546AE
:1000C00000F032FC004800471D36000818070020E9
:1000D0000C4880F308880C480168090E0B4A9142CD
:1000E00005D10B480B4901600B480C4901600C48D5
:1000F00080470C480047FEE7FEE7FEE7FEE7FEE725
:10010000FEE7000018070020040000001F000000A8
:100110001810024001000000000001400000000033
:1001200019220008BD00000830B50B46014600202A
:100130002022012409E00D46D5409D4205D31D46ED
:100140009540491B2546954040191546521E002DE5
:10015000F1DC30BD70B500242546002801DA012409
:100160004042002901DA01254942FFF7DDFFAC4298
:1001700000D04042002C00D0494270BD30B5054649
:100180000020034600E05B1C934205D2EC5CC85C97
:10019000201A01D1002CF6D130BDF8B502464A40F4
:1001A000D40F42004B0052085B089A4202D202462A
:1001B000084611464A0023D0C30D4A00DDB2120E94
:1001C000AD1A202D35DA49020126490AF6058A19A9
:1001D000002C00D0524220214F1B1146B9402A4129
:1001E0001018C20D9A4221D0002C17D0012D08DC26
:1001F000DA05801AD20F8019D207DBB200F0AEF90F
:10020000F8BDDA05801A012340001B06C0188018CB
:100210005A428018CA0F1043490007E04908C20734
:100220001143DA05801A80194008801800F08EF911
:10023000F8BD61000122511A001BF7E70122D20725
:100240005140AAE70122D2075040A6E7024670B506
:100250004A40D30FDB0740002DD04A002AD0010EC0
:10026000140E000212020919400A520A8418E5010C
:1002700004465443000A120A2E045043A41942199A
:10028000200CC543AA18120C0125AD03521C5219AB
:1002900012047F39240400D0521C104301D44000C2
:1002A000491EC2B20C06C0092018401C4008802A12
:1002B00002D003E0002070BD40084000002900DAB1
:1002C0000020184370BD70B502464A40D50F40006B
:1002D0004A00ED0740085208002814D0002A12D026
:1002E000C40DD30D41020120C0055202490A520A31
:1002F000E41A091812187D34914201D3641C00E0FD
:100300004900002C01DA002070BD0023914201D386
:10031000891A0343400849000028F7D100290AD070
:10032000914202D10121C90705E0914201D2012188
:1003300001E00121C943E005C018401900F006F9A9
:1003400070BD0000F0B50C465C4085B0E40FE407DA
:1003500003944C000026640859009446490802465C
:100360000296224321D062460A431ED06200570DF6
:100370004A000E032303550D012402462C4924058F
:10038000781B1B0B360B4018234326436146009015
:100390001C46501AB44103D30098401C009002E060
:1003A000921800985B41002803DA0020014605B04E
:1003B000F0BD0020012109050746864611E064468C
:1003C0001D46141BB54106D36546521BB341744606
:1003D00007430C43A646CD07400849082843921816
:1003E0005B4105460D43EAD11046184313D06046E1
:1003F000194650407140084306D06046101AB34178
:1004000006D20122002306E000220123DB0702E0DE
:100410000122D2435310009874460105381C6141F3
:10042000029C039D0019694100F0D1F8BFE700006C
:10043000FD03000010B500229623114600F08EF84F
:1004400010BD00000EB5C217C10F5040CA074018BA
:100450000021054B0293019200910A460B4600F0E1
:10046000C3F803B000BD000033040000C20F410018
:1004700040020123400ADB05D207090EC0187F297C
:1004800001DA00207047962903DC9623591AC840E8
:1004900001E096398840002AF4D040427047CB0FE3
:1004A000DB07490010B5490802460A4307D00A0D88
:1004B00007240903E401090B121B002A01DC0020B8
:1004C00010BDC900440F0C43C100E018D2058018CC
:1004D00000F03CF810BD00000122D207002800DB2C
:1004E000101A002900DB511A88427047F0B51FB47A
:1004F0000646002082B005464024019100901BE092
:10050000019922460F46304600F030FA049A059BC6
:10051000801A994110D310461946224600F016FA67
:10052000361A8F410197224601200021009F00F0DA
:100530000DFA38184D4100902046641E0028DFDC7B
:10054000019B00982946324607B0F0BD002904DA25
:10055000401C490001D140084000704770B400249D
:10056000050C05D11024000402D1002921D011244A
:10057000050E01D100020834050F01D10001241D30
:10058000850F01D18000A41C002801DB4000641C01
:10059000002908D020252E1B0D46F540A14000D093
:1005A00001212943084301061B1B000ADB1D02D55C
:1005B000002070BC7047DB05181880180029F8DA95
:1005C000401C4900F5D170BC40084000704710B590
:1005D000002B08DA0024401C614192185B411A4349
:1005E00001D14008400010BDF0B51FB482B00546EF
:1005F0000C0003D0084602F083FB02E002F080FB0F
:100600002030024600902146284600F09FF9049BC6
:10061000059A04460F4618431143084314D0184660
:1006200010431BD0009840210A1A1846059900F083
:100630009DF905460E46009A0599049800F086F942
:10064000084305D0012004E02046394607B0F0BD3C
:100650000020C11705430E432C43374300990E98E1
:100660006305401A7905E40A00220C43FD0A0A30AA
:1006700002D500200146E9E70105101969410C9CEB
:100680000D9D00196941FFF7A2FFDFE7F0B50746AE
:100690000846584087B0C00F049048000E465900E5
:1006A00040084908BC1A884105D2384631461E46E2
:1006B00017460B4602465800400810434CD0300DF8
:1006C000039040055900400D490D0590401A0290D5
:1006D000402872DA18030121000B09050843019034
:1006E00004980092002805D00199524200208841C8
:1006F00000920190029840210A1A0199009800F096
:1007000025F905460C466B4607CB00F040F9C019A9
:100710007141039A0E0D0023D71756401A467A40AE
:10072000164344D0049A002A2DD0029A012A039A33
:1007300015DC1205C01A914101263605001C7141D5
:10074000D20F059ED2070093019202962A462346B5
:10075000FFF74AFF07B0F0BD38463146FAE7160505
:10076000224A0F46B218C01AB74101210905001CE0
:100770004F4100187F41114618187941E20F10438C
:100780006D19644113E0E2076D0815436408C20760
:100790001443039A01261205C01A91413605001C24
:1007A0007141CE07400830434908C01851412A46DC
:1007B0002346FFF70CFFCDE7FFE704980122400036
:1007C000C117121A00238B4104983146C417381AF6
:1007D000A141EEE730B40124E407634030BC55E7A3
:1007E00030B40124E407614030BC4FE70000E0FF73
:1007F000F0B51FB488B00B990998002448400999B6
:10080000C00F490049080991C0070B9900904900A1
:1008100049080B9109990898A64608431CD00B99E2
:100820000A98084318D0099801244000420D480056
:10083000410D099824050003000B204309900B98F3
:100840000003000B20430B9050181C494018002255
:1008500001901446104605E0002001460DB0F0BDA1
:10086000032801DA034600E003239C46C11A0AAEBE
:100870000AE05F0008ADED5B4F00F75B7D430027AA
:10088000AA187C41491C5B1E6145F2DD410004ABA6
:100890005A522104120C0A43240C401C0828DFDBA6
:1008A000019802900099704601910090059B049A6E
:1008B00007990698FFF798FED0E700000DFCFFFFB0
:1008C0004A0009030123090B1B0519430A4B10B504
:1008D000520D9A4202DA0020014610BD064B343315
:1008E0009A4203DC9A1A00F041F810BD034BD2186B
:1008F00000F02CF810BD0000FF030000CDFBFFFF4F
:1009000010B5002904DB0124E40740428C41214654
:10091000002B04DB1C460123DB075242A341994212
:1009200000D1904210BD0000064C0125064E05E0A6
:10093000E36807CC2B430C3C98471034B442F7D300
:10094000FFF7C0FB183800083838000810B5202A17
:1009500004DB0146203A9140002010BD9140202345
:100960009C1A0346E3401943904010BD10B5202A5D
:1009700004DB0846203AD040002110BD0B46D3408E
:10098000D0402024A21A91400843194610BD10B54A
:10099000202A06DBCB170846203A1041C1170B432B
:1009A00006E00B461341D0402024A21A9140084390
:1009B000194610BDFFB587B00446109D0021206880
:1009C000FFF78AFD03D801212420015502E0002110
:1009D000242001552068FFF749FDC1B225200155AB
:1009E0008A492068FFF732FC0290FFF73FFD64213F
:1009F0000390FFF7AFFB262001550026012004E0FD
:100A00000899095C8919CEB2401C0828F8DBF0432C
:100A1000401CC6B20898007A864212D1089989789B
:100A20000A020899C9785018FFF70CFD0022784B8C
:100A300001910090FFF786FC03910290FFF72FFDD4
:100A4000A0600027012004E00A99095CC919CFB20F
:100A5000401C0828F8DBF843401CC7B20A98007A0B
:100A6000874212D10A9989790A020A99C9795018DC
:100A7000FFF7E8FC0022674B01910090FFF762FC52
:100A800003910290FFF70BFD20610020059000BF4D
:100A900005E02A5C0599511889B20591401C1D2872
:100AA000F7DB05980012A97F88421CD10598C0B2D7
:100AB000E97F884217D1287B0002697B4018E061FA
:100AC000A87B0002E97B401820627D210901E069D2
:100AD000884201DD0846E0617D210901206A8842E3
:100AE00001DD0846206200200490012006E00999FB
:100AF0000A5C04995118C9B20491401C0828F6DB1D
:100B00000498C043401CC0B204900999097A049823
:100B1000884212D1099989780A020999C97850182E
:100B2000FFF790FC00223A4B01910090FFF70AFC7E
:100B300003910290FFF7B3FCE0606068FFF796FC5A
:100B4000C1B22720015531496068FFF77FFB029051
:100B5000FFF78CFC64210390FFF7FCFA2820015575
:100B6000A068FFF783FCC1B2292001552749A0687E
:100B7000FFF76CFB0290FFF779FC64210390FFF70D
:100B8000E9FA2A200155E068FFF770FCC1B22B207A
:100B900001551E49E068FFF759FB0290FFF766FC1C
:100BA00064210390FFF7D6FA2C2001552069FFF746
:100BB0005DFCC1B22D20015514492069FFF746FBA9
:100BC0000290FFF753FC64210390FFF7C3FA2E2035
:100BD0000155A08A0004010E2F200155217D3020EF
:100BE0000155207EA061A08B0004010E3320015529
:100BF000217F34200155208C0004010E3520015541
:100C0000208CC1B2362001550BB0F0BD0000C842A7
:100C10000000594000408F4010B500F001F810BDB1
:100C200010B502A002F05CF810BD000041542B5337
:100C300054415455533D3F0D0A00000010B50120AA
:100C4000400200F023F80120400200F001F810BD3E
:100C5000012109070140002902D00349486001E051
:100C60000249486070470000000402400000024052
:100C7000002904D0026801231A43026003E00268DD
:100C8000014B1A4002607047FEFF00000146002041
:100C9000002201231B070B40002B02D0064B1A68D1
:100CA00001E0064B1A6813460B40002B01D00120CF
:100CB00000E00020704700000004024000000240F5
:100CC00010B5002202680D4B1A400C6A8B68234352
:100CD0000C6923434C6923438C692343CC69234328
:100CE0004C6A23438C6A23431A430260CB684360F7
:100CF0000B6883604B68C36010BD00000F80FFFF6E
:100D000010B50B4A904200D100E000BFA822125853
:100D10000B0F9C000F23A3409A43A8231A50A8222C
:100D200012580B011B091A43A8231A5010BD0000CA
:100D3000000002401CB5084800F03CFA074808498A
:100D4000084B094A0091019008490348FFF732FE19
:100D5000014801F06DF91CBD5C000020D4010020A9
:100D600014010020D40000209401002094000020F1
:100D70000349086000BF024909680029FBD1704798
:100D80003C0000200EE00021084A116005E000BF91
:100D900006490968491C054A116004490968042983
:100DA000F5D3401E0028EED170470000400000201F
:100DB0000FE00021084A116005E000BF06490968FC
:100DC000491C054A116004490968044A9142F4D358
:100DD000401E0028EDD17047440000200B11000098
:100DE00010B5012000F016F8002805D001200449B4
:100DF000087000F009F802E003200249486110BDC4
:100E0000540000200004014001494861704700007F
:100E10000004014001460020044A52690A40002AA9
:100E200001D0012000E000207047000000040140D4
:100E3000002806D00649096810221143044A1160AF
:100E400005E00349096810229143014A1160704787
:100E50000020024001460020044A1068400840007B
:100E600002460A431046014A1060704700200240C3
:100E70001CB5012203210920C00600F06BF90122F4
:100E800002210920C00600F065F90C200090022123
:100E9000684601710321417100218171C171694668
:100EA0000920C00600F00EF900220721824800F058
:100EB00051F900220621804800F04CF9C020009032
:100EC0000221684601710321417100218171C171C4
:100ED0006946794800F0F6F801220521774800F0CC
:100EE00039F901220421754800F034F930200090CE
:100EF0000221684601710321417100218171C17194
:100F000069466E4800F0DEF8042201210920C0067F
:100F100000F020F9042200210920C00600F01AF98F
:100F200003200090022168460171032141710021D4
:100F30008171C17169460920C00600F0C3F8022220
:100F400011465F4800F006F902220C215B4800F0D0
:100F500001F90420009002216846017103214171CA
:100F600000218171C1716946554800F0ABF801203C
:100F700000030090022168460171032141710021A4
:100F80008171C17169464D4800F09CF805221146F7
:100F90000920C00600F0DEF8052204210920C00661
:100FA00000F0D8F83020009002216846017103213A
:100FB000417100218171C17169460920C00600F0AC
:100FC00081F8012207213D4800F0C4F801220621E2
:100FD0003A4800F0BFF8C020009002216846017135
:100FE0000321417100218171C1716946334800F0CC
:100FF00069F801220921314800F0ACF801220821EA
:101000002E4800F0A7F80320000200900221684655
:1010100001710321417100218171C1716946274825
:1010200000F050F803208002009000216846017112
:101030004171C1716946204800F044F8FF20013039
:101040000090012168460171002141710121C171A7
:101050000021817169460920C00600F033F80C2098
:101060000090012168460171002141710121C17187
:10107000002181716946114800F024F804210F48CD
:1010800000F096F808210D4800F092F80120C00306
:101090000090012168460171002141710121C17157
:1010A000002181716946044800F00CF80121C90350
:1010B000014800F07DF81CBD00040048000800480D
:1010C000000C0048F0B50A4600210023002400BFB0
:1010D0003DE001258D402B4615681D402C469C4265
:1010E00034D11579012D02D01579022D16D18568DC
:1010F0004F000326BE40B543856055794E00B5408C
:10110000866835438560858801268E40B543858095
:10111000858896798E40B6B23543858005684F0044
:101120000326BE40B543056015794E00B5400668FC
:1011300035430560C5684F000326BE40B543C56012
:10114000D5794E00B540C6683543C560491C1029A5
:10115000BFD3F0BDF0B5002300244D07EE0E1546B9
:10116000B5402B46CD10AE0005462035AD594E0793
:10117000F70E0F26BE40B543CE10B6000746203707
:10118000BD51CD10AE003D46AD591D432C46CD108E
:10119000AD003E467451F0BD02460020138A0B405C
:1011A000002B01D0012000E000207047018570472E
:1011B0008161704738B50446C820FFF7D9FD012189
:1011C00089024548FFF7E8FF312108550121C9028E
:1011D0004148FFF7E1FF322108553120005D00282A
:1011E00001D1012000E000203221095D002901D158
:1011F000012100E000210840002801D00020A0616A
:101200003120005D002801D1012000E000203221C2
:10121000095D012900D100E000210840002801D02B
:101220000120A0613120005D012800D100E00020F4
:101230003221095D002901D1012100E0002108408F
:10124000002801D00220A0613120005D012800D1DA
:1012500000E000203221095D012900D100E00021D9
:101260000840002801D00320A061C820FFF780FDBE
:1012700007221A491A4801F01DFDC820FFF778FD22
:1012800009221849184801F015FDC820FFF770FD24
:1012900009221649164801F00DFDC820FFF768FD28
:1012A00009221449144801F005FDC820FFF760FD2C
:1012B00009221049114801F0FDFC3220FFF778FDAA
:1012C000322001230022211D0090204600F003FD62
:1012D0003220FFF76DFD38BD0004004838370008A4
:1012E000004C00405B370008001401409A370008AA
:1012F000004800407F37000800500040003801409F
:1013000000BFFEE7F8B504460E46174600200090E1
:101310002070012080020921C9068861802522E011
:10132000012040020921C90688610120FFF72AFD3A
:10133000384600F082F800900320FFF723FD0920D3
:10134000C006008A012189020840002802D02078C6
:1013500028432070012040060921C9068861012028
:10136000FFF710FD6D10002DDADC002E05D10120F5
:1013700080060921C906886104E001208002092154
:10138000C90688610120FFF7FDFC01204002092108
:10139000C90688610520FFF7F5FC012040060921F8
:1013A000C9068861C01388611420FFF7EBFC009820
:1013B000F8BD10B5012080020921C906886101200D
:1013C000FFF7E0FC012040020921C90688610120E5
:1013D000FFF7D8FC012080060921C90688610A2090
:1013E000FFF7D0FC012040060921C90688610A20C8
:1013F000FFF7C8FC10BD10B5012040060921C90641
:1014000088610120FFF7BEFC012080060921C90682
:1014100088610120FFF7B6FC012040020921C906BE
:1014200088610A20FFF7AEFC012080020921C9066D
:1014300088610A20FFF7A6FC10BD70B504460025A0
:1014400009E02046611ECCB2002801D1042070BD05
:101450000120FFF7ADFC0920C006008A01214902E6
:1014600008400028EDD02846F1E770B50546002673
:10147000802422E020462840002805D10120800653
:101480000921C906886104E0012080020921C906FA
:1014900088610120FFF776FC012040020921C9067E
:1014A00088610520FFF76EFC012040060921C9066E
:1014B00088610120FFF766FC6410002CDADC012053
:1014C00080020921C9068861401088610120FFF768
:1014D00059FC0920C006008A012189020840002821
:1014E00000D00126012040060921C9068861142088
:1014F000FFF748FC304670BD70B505460C460748FE
:1015000000F02EF8284600F01FF8204600F022F8E0
:1015100000F012F800F004F870BD0000555500000E
:101520000148024908607047CCCC00000030004000
:1015300010B500F001F810BD01480249086070477D
:10154000AAAA00000030004001494860704700002E
:1015500000300040014988607047000000300040C2
:10156000014908607047000000300040704708B52E
:101570001C216846017001214170817000F03AF829
:101580001B216846017001214170817000F032F822
:101590001D216846017001214170817000F02AF818
:1015A0001D216846017001214170817000F022F810
:1015B0001D216846017001214170817000F01AF808
:1015C0001D216846017001214170817000F012F800
:1015D0001D216846017001214170817000F00AF8F8
:1015E0001D216846017001214170817000F002F8F0
:1015F00008BD000000218278002A27D0184A032362
:101600001B02D21803789B109B00D15802789207D6
:10161000D30EFF229A400B46934319464278920715
:10162000120E03789B07DB0E9A4011430C4A0323EA
:101630001B02D21803789B109B00D1500278D3066E
:10164000DB0E01229A40064B1A6007E00278D306AF
:10165000DB0E01229A40024B80331A607047000073
:1016600000E100E010B5002819DA1A4A03071B0F41
:10167000083B9B089B00D2588307DC0EFF23A34046
:101680009A438B071B0E8407E40EA3401A43114BA9
:101690000407240F083CA408A4001A5118E00E4ABD
:1016A00003231B02D21883089B00D2588307DC0E49
:1016B000FF23A3409A438B071B0E8407E40EA3402D
:1016C0001A43054B032424021B198408A4001A5151
:1016D00010BD00001CED00E000E100E010B5034883
:1016E0000078032801D100F003F810BD2400002089
:1016F00010B502A001F0F4FA10BD000041542B43D4
:10170000555252454E5444523D350D0A00000000DA
:1017100070470000002905D0054A52690243044B76
:101720005A6104E0024A52698243014B5A61704790
:1017300000100240002905D0054AD2690243044B3B
:10174000DA6104E0024AD2698243014BDA617047F0
:1017500000100240002905D0054A92690243044B5B
:101760009A6104E0024A92698243014B9A61704790
:101770000010024019480068012108431749086019
:101780000846406816490840144948600846006801
:10179000144908401149086008460068012189047D
:1017A00088430E490860084640683F210904884381
:1017B0000A4948600846C06A00090001C862084634
:1017C000006B09490840054908630846406B40081A
:1017D000400048630020886070470000001002400D
:1017E0000CB8FF08FFFFF6FEACFEF0FFFEB50446A6
:1017F00000250026002002900190009000278648D6
:1018000040680C2108400546002D06D0042D07D065
:10181000082D08D00C2D2CD128E0804820602BE02A
:101820007F48206028E07C4840680F2189040840F8
:101830000646794840680321C90308400290B00C6D
:10184000861C0298002803D17648374647430BE0B0
:101850007148C06A0007000F401C01907048019950
:10186000FEF762FC70430746276005E06E48206083
:1018700002E06A48206000BF00BF67484068F0216E
:10188000084005462D096948405D00902068009990
:10189000C84060606048406807210902084005466A
:1018A0002D0A6248405D009061680098C140A160C7
:1018B0005948006BFF2101310840884202D05C4842
:1018C000E0600DE0544840680121890308408842E7
:1018D00003D0A0684008E06002E0A0688008E060F3
:1018E0004D48006B40210840402802D051482061FB
:1018F00002E00120C00320614748006B102108402E
:10190000102802D04548606101E0206860614248CB
:10191000006B8007800F002802D1A068A06119E049
:101920003D48006B8007800F012802D12068A0612C
:1019300010E03948006B8007800F022802D1800335
:10194000A06107E03448006B8007800F032801D1B5
:101950003248A0613048006B032109040840002888
:1019600002D1A068E06120E02B48006B032109044C
:10197000084001210904884202D12068E06114E096
:101980002548006B032109040840012149048842CD
:1019900002D18010E06108E01F48006B03210904B8
:1019A0000840884201D11D48E0611B48006B0321BB
:1019B00089040840002802D1A068206220E016486F
:1019C000006B03218904084001218904884202D167
:1019D0002068206214E01048006B0321890408404D
:1019E0000121C904884202D10011206208E00A489E
:1019F000006B032189040840884201D10748206216
:101A00000548006B80210840802802D006486062AB
:101A100000E06762FEBD00000010024000127A0084
:101A20000024F40000093D00006CDC0214000020DA
:101A3000809FD5001280000010B5024600210023CF
:101A400000205111002902D10C4C23680BE0012920
:101A500002D10A4C236A06E0022902D1074C636ACC
:101A600001E0064C636BD106C90E01248C401C407A
:101A7000002C01D0012000E0002010BD0010024029
:101A8000024840680C2108407047000000100240E6
:101A900001460020054A5068F02302469A4310464A
:101AA00002460A431046014A506070470010024047
:101AB0000021024A91701146887070470010024060
:101AC0000549096B10229143034A11631146096BC2
:101AD00001431163704700000010024001460020DE
:101AE000064A506807231B0202469A4310460246E4
:101AF0000A431046014A506070470000001002403F
:101B0000002807D007490968012212061143054A37
:101B1000116006E003490968012212069143014A57
:101B20001160704700100240074A52687B23DB03B4
:101B30009A43054B5A601A46526803460B431A43B0
:101B4000014B5A607047000000100240014600201F
:101B5000044AD06A0009000102460A431046014ABD
:101B6000D06270470010024001460020044A5068CD
:101B70008008800002460A431046014A50607047C0
:101B8000001002400021010F012906D10E4A126BFC
:101B9000920892000C4B1A6310E0022907D10A4AFE
:101BA000126B03231B049A43074B1A6306E0064A91
:101BB000126B03239B049A43034B1A63024A126B72
:101BC0000243014B1A637047001002400549096B3C
:101BD00080229143034A11631146096B014311634B
:101BE000704700000010024038B50020009000242B
:101BF000002500BF1120FFF71FFF05460098401C7D
:101C00000090052109030098884201D0002DF1D0F1
:101C10001120FFF711FF002801D0012400E000246B
:101C2000204638BD70B502460B46FF20002115E066
:101C3000555C684008240DE080250540002D05D046
:101C40004500FF2632367540E8B201E04506280E11
:101C5000651EECB2002CEFDC4D1CE9B29942E7DBCB
:101C600070BD000070B504462046FEF7E3FB064653
:101C70000349FEF7EBFA05460249FEF724FB70BD67
:101C80000000C84200FF7F47F8B504462046FEF733
:101C9000D1FB07460549FEF7D9FA06460449FEF787
:101CA00012FB05460349FEF7C9FAF8BD00002F43B1
:101CB00000FF7F4700003442F8B505460E46144643
:101CC00031462846FFF7AEFF0746A74201D0022063
:101CD000F8BD0020FCE7FFB581B006460F461D4663
:101CE000002D02D0012D10D107E0394630460A9B65
:101CF000039A00F011F8044609E0394630460A9B81
:101D0000039A00F055F8044601E0802400BF00BFAC
:101D1000204605B0F0BD0000FFB583B005460E4675
:101D2000174600F02BF90446002C19D1002F0ED0D5
:101D3000012F06D0022F10D11C4800F02FF90446C5
:101D40000DE01A48C01E00F029F9044607E01748C4
:101D50000A3800F023F9044601E0802400BF00BFE8
:101D6000002C02D100F0FEF80446002C05D1002121
:101D700002A8069A00F0BAF80446002C05D1002209
:101D8000012101A800F0B2F8044600F003F9002C8C
:101D900009D168460089FFF777FF28606846808888
:101DA000FFF760FF3060204607B0F0BD102C000048
:101DB000FFB583B006460F461D4600F0DFF8044627
:101DC000002C1AD1059800280ED0012806D0022830
:101DD00010D1244800F0E2F804460DE021480B3809
:101DE00000F0DCF8044607E00920800200F0D6F895
:101DF000044601E0802400BF00BF002C13D109E09D
:101E000000F0B0F80446002C00D108E07D20C000AE
:101E1000FEF7B8FF2846691ECDB20028F0D100BFFA
:101E2000002D00D10424002C0BD10022114602A861
:101E300000F05CF804430022012101A800F056F8EC
:101E4000044300F0A7F8002C09D168460089FFF789
:101E50001BFF306068468088FFF704FF386020462B
:101E600007B0F0BD162400001CB504460120800216
:101E70000090002168460171C17169461A48FFF758
:101E800021F9012000030090012168460171002121
:101E90008171032141710021C17169461248FFF728
:101EA00011F9012040071049886103204002009089
:101EB0000121684601718171032141710021C171C5
:101EC00069460920C006FFF7FDF8012080020921BC
:101ED000C906886140108861204600F033F801206F
:101EE0004003014988611CBD00040048FEB5054659
:101EF0000E4617463A46002101A8FFF703FA0446AA
:101F0000002C06D10022114601A80130FFF7FAF992
:101F10000446002C05D1002231466846FFF7F2F94D
:101F20000446002C06D168460278022101A8FFF77A
:101F3000C3FE0446694608790002497908432880AF
:101F40002046FEBD4106090E044A1170114609786B
:101F500001221143024A1170704700002B0000203B
:101F60002C00002010B5FFF724FA03480078FFF793
:101F70007CFA0446204610BD2C00002010B5FFF767
:101F800018FA03480078FFF770FA0446204610BD9F
:101F90002B00002010B5FFF72EFA10BD70B50446D7
:101FA0002012FFF762FA0546E0B2FFF75EFA05433A
:101FB000284670BD7047000010B590B0044636202A
:101FC000005D3521095D3422125D33231B5D0B93C7
:101FD0000C920D910E903021095D2F22125D2E235F
:101FE0001B5DA0690793089209910A902D20005D5E
:101FF0002C21095D2B22125D2A231B5D0393049281
:10200000059106902920015D2820005D2722125DA0
:102010000092029101902620035D2520025D24207C
:10202000015D024800F05CFE10B010BDB83700083A
:1020300010B5044603480078032802D12046FFF774
:10204000BBFF10BD2400002010B5C820FEF790FE95
:1020500007221749174800F02DFEC820FEF788FE1A
:1020600009221549154800F025FEC820FEF780FE1C
:1020700009221349134800F01DFEC820FEF778FE20
:1020800009220F49104800F015FEC820FEF770FE27
:1020900009220E490E4800F00DFE6420FEF788FE6E
:1020A0004420FFF7E1FE3220FEF782FE10BD000063
:1020B0003F370008004C0040A337000800480040AC
:1020C000883700080050004000380140643700089D
:1020D000001401400CB500200190009031480068C8
:1020E0000121090408432F49086000BF2D480068FA
:1020F00001214904084000900198401C019000987B
:10210000002804D10521090301988842EED1254811
:102110000068012149040840002802D001200090F5
:1021200001E0002000900098012839D111201E49BB
:1021300008601C4840681B49486008464068486081
:10214000084640687F21C90388431649486008460D
:1021500040680521090408431249486008460068A0
:102160000121090608430F49086000BF0D480068B7
:102170000121490608400028F8D00A484068800834
:102180008000084948600846406802210843054924
:10219000486000BF034840680C2108400828F9D176
:1021A0000CBD0000001002400020024010B57D214F
:1021B000C90010480068FDF7B7FF0446601E0E49CD
:1021C000884201D901200CE0601E0C4948610321BE
:1021D000081FFFF747FA00200849886107200861B7
:1021E0000020002801D000BFFEE70021481EFFF7B5
:1021F00039FA10BD00000020FFFFFF0000E000E002
:1022000004480068002804D002480068401E0149C4
:10221000086070473C00002010B51B480068012191
:10222000084319490860084640681849084016499B
:102230004860084600681649084013490860084687
:1022400000680121890488430F49086008464068F6
:102250003F21090488430C4948600846C06A0009C8
:102260000001C8620846006BFF21543188430649CB
:1022700008630846406B40084000486300208860BF
:10228000FFF728FF10BD0000001002400CB8FF0847
:10229000FFFFF6FE10B50121134800F03FF80028BB
:1022A00020D00121104800F028F8104800780028BC
:1022B00009D001280ED0022813D101200B49087043
:1022C0000B4908700DE002200849087001200849F8
:1022D000087006E0002005490870012004490870D4
:1022E00000BF00BF10BD000000100040250000200E
:1022F00026000020CA4302827047CA430282704708
:10230000002904D0028801231A43028003E00288D6
:10231000014B1A4002807047FEFF000030B50246B4
:10232000002000230024158A0D402B4695890D407E
:102330002C46002B03D0002C01D0012000E000200F
:1023400030BD002A03D083890B43838102E0838957
:102350008B438381704700000EB501211020FFF7E9
:10236000E9F90B4801900B48694608800A4800F0DB
:1023700015F801210848FFF7BDFF01221146064864
:10238000FFF7DFFF01210448FFF7BAFF0EBD000091
:10239000BF5D00001F4E00000010004000220288B8
:1023A000154B984206D001239B07984202D0134B4D
:1023B000984203D1124B1A404B881A43114B984252
:1023C00003D0114B1A400B891A4302804B68C36239
:1023D0000B880385084B984208D00C4B984205D0D7
:1023E0000B4B984202D00B4B984201D18B7A03865B
:1023F0000123838270470000002C0140000400404C
:102400008FFF000000100040FFFC00000040014072
:10241000004401400048014010B500F003F8FFF708
:102420009BFF10BD08B51121684601700021417065
:1024300001218170FFF7DEF808BD000010B50B49DF
:102440000B4800F0B9FA00280FD00849084800F0FE
:10245000BBF900210748FEF70BFC4020054908396D
:10246000C86001210348FEF703FC10BD040104000D
:10247000003801400800024010B50749074800F045
:102480009BFA002807D0054800F06CFBC4B2024953
:10249000024800F099F910BD050105000044004014
:1024A00010B5AD49AD4800F087FA00280FD0AA4911
:1024B000AA4800F089F90021A948FEF7D9FB40207D
:1024C000A749303948630121A548FEF7D1FBA2494D
:1024D000A44800F071FA00280FD09F49A14800F0ED
:1024E00073F90021A048FEF7C3FB80209E491C39E8
:1024F000086201219C48FEF7BBFB97499B4800F00E
:102500005BFA002811D09449984800F05DF9002149
:1025100093482830FEF7ACFB402091491031C86148
:1025200001218F482830FEF7A3FB9149914800F024
:1025300043FA002812D08F4800F014FB8E498F4ACE
:10254000127888548D480078401C8C4908700846E1
:10255000007808708649874800F036F98748007887
:10256000401E8549085CFF2805D184480078401E3C
:10257000834908704EE081480078401E8049097800
:10258000491C88420CD17D480078401E7A49085C7D
:10259000862805D179480078401E7A49087039E0CC
:1025A00076480078401E77490978C91D884231D1A4
:1025B0000020744A117804E06F4A525C1218D0B2BD
:1025C000491C704A1278D21D9142F5DBC143491C67
:1025D000C8B2694A6B490978C91D515C884213D158
:1025E0001146684A1278895C86290DD1624A65498C
:1025F0000978491C515C0A025F4B62490978891CC1
:10260000595C5118604A51610021604A11705B4A5F
:10261000117000BF56495E4800F0CEF9002815D071
:1026200053495B4800F0C8F900280ED0584800F024
:1026300099FAC4B200BF8021564800F0B3F90028CF
:10264000F9D04B49524800F0BFF800BF4249524808
:1026500000F0B2F900287ED03F494F4800F0B4F8AE
:10266000002141481430FEF703FB80203E491C390D
:10267000486301213C481430FEF7FAFA0A22474920
:1026800047A0FDF77BFD00281CD14448807A3038F4
:10269000002806D0012808D002280AD0032810D12B
:1026A0000BE00020414908700BE001203F49087011
:1026B00007E002203D49087003E003203B49087011
:1026C00000BF00BF0A22354939A0FDF757FD002899
:1026D0001CD13248807A3038002806D0012808D032
:1026E00002280AD0032810D10BE000202F490870DF
:1026F0000BE001202D49087007E002202B490870EB
:1027000003E003202949087000BF00BF08222349C5
:102710002AA0FDF733FD00281DD12048007A30386B
:10272000002806D0012809D002280BD0032811D197
:102730000CE000201D4908700CE00CE001201B4952
:10274000087007E002201949087003E003201749C8
:10275000087000BF00BF10BD040104000048004025
:1027600030000240004C00401C0402400050004079
:102770000501050000140140D401002027000020BD
:1027800028000020290000205C0000202A000020F2
:102790000018014000440040001C01409402002049
:1027A0000D0A2B5354415455533A00002400002085
:1027B0000D0A5E5354415455533A00005E53544140
:1027C0005455533A0000000010B5002300220B0CB2
:1027D00001249C402246026210BD002904D00268F8
:1027E00001231A43026003E00268520852000260AB
:1027F0007047000000B587B0E12040020190002042
:1028000002900390049006900C20059001A957486F
:1028100000F01AF900225649544800F0F4F801215A
:102820005248FFF7DAFF4B20C001019000200290D0
:102830000390049006900C20059001A94D4800F0EB
:1028400003F900224A494B4800F0DDF801214948CC
:10285000FFF7C3FF4B20C0010190002002900390BE
:10286000049006900C20059001A9434800F0ECF874
:1028700000223F49404800F0C6F801213E48FFF7DA
:10288000ACFF4B20C0010190002002900390049007
:1028900006900C20059001A9384800F0D5F80022D8
:1028A0003349364800F0AFF801213448FFF795FF6F
:1028B0004B20C001019000200290039004900690EC
:1028C0000C20059001A92E4800F0BEF800222849EE
:1028D0002B4800F098F801212948FFF77EFF4B2094
:1028E000C0010190002002900390049006900C20FB
:1028F000059001A9234800F0A7F801221C492148AE
:1029000000F081F801211F48FFF767FFE120400236
:102910000190002002900390049006900C200590F6
:1029200001A9194800F090F801221149164800F059
:102930006AF800211448FFF750FF4B20C0010190B6
:10294000002002900390049006900C20059001A9AD
:102950000E4800F079F8002205490C4800F053F8C1
:1029600001210A48FFF739FF07B000BD00440040CD
:10297000050105000038014000480040004C0040BF
:10298000005000400014014000180140001C0140AC
:10299000002A03D083680B43836002E083688B4383
:1029A0008360704702460020D3690B40002B01D0A2
:1029B000012000E00020704770B502460B4600245D
:1029C0000021002500201E04350ED9B201268E40BC
:1029D0003146012D02D11668314006E0022D02D1A8
:1029E0005668314001E0966831401C0C0126A64033
:1029F0003446D6693440002903D0002C01D0012090
:102A000000E0002070BDF8B50346002400260096C3
:102A10000025002018460E04340ECEB20096012781
:102A2000009EB7403D46022C01D1001D02E0032C60
:102A300000D10830002A03D006682E43066002E069
:102A40000668AE430660F8BDF0B58BB004460D468F
:102A5000002700200A9000262068400840002060DF
:102A6000666803210903304688430646A868064382
:102A7000666026682D480640E96868680843296949
:102A8000084306432660A6680321090230468843AE
:102A9000064668690643A6606846FEF7A7FE244816
:102AA000844202D106980A900DE02248844202D165
:102AB00007980A9007E02048844202D108980A90BB
:102AC00001E002980A9020680121C903084000280B
:102AD0000CD029680A9A5000FDF726FB07462968A2
:102AE0000A9A5000FDF720FB0E4609E029680A9873
:102AF000FDF71AFB074629680A98FDF715FB0E46F5
:102B000028684008B04200D87F1C20680121C90312
:102B10000840002806D03807460F384607490840C5
:102B200030430746A7810BB0F0BD0000F3E9FFFF7B
:102B3000003801400044004000480040F0FF000021
:102B400010B501212F204004FEF7E4FD01210F20E4
:102B50004004FEF7EFFD01210148FEF7FBFD10BD2B
:102B6000E14000000146888CC005C00D7047CA05D1
:102B7000D20D0285704700000EB508202049402282
:102B8000204B0092019102901F4A01211C480830FD
:102B900000F056F81D481A4940221D4B0092019141
:102BA00002901C4A01211648303000F049F81A48BA
:102BB0001A4980221A4B009201910290194A02216F
:102BC00016481C3000F03CF817480D494022174BBE
:102BD000009201910290164A01210948583000F0F4
:102BE0002FF814480D498022134B00920191029056
:102BF000124A02210948303000F022F80EBD0000D0
:102C0000000002409400002000380140000A00202B
:102C1000D400002000480040B00000100004024032
:102C200014010020004C004000000C4094010020E2
:102C300000500040000F002094020020001C0140C2
:102C4000F0B58BB007460D4614461E4601212846B6
:102C5000FEF760FD2046243000900196002002908F
:102C6000109803900020049080200590002006908A
:102C70000790089001200003099000200A906946FF
:102C80003846FEF71DF801213846FDF7F1FF12998D
:102C90001198FEF735F8012205492046FFF7B3FEEB
:102CA000012240212046FFF773FE0BB0F0BD00006B
:102CB0000401040070B506460C4615460BE0217869
:102CC000641C3046FFF753FF00BF80213046FFF7FA
:102CD00069FE0028F9D028466D1E0028EFD170BD8E
:102CE0000FB410B503A9044B044A029800F0E8F8A9
:102CF00010BC08BC04B01847F93500085800002083
:102D00002021020C01D010211046020A01D01046E9
:102D10000839020901D01046091F820801D0104667
:102D2000891E420801D0881E7047081A704702E0C9
:102D300008C8121F08C1002AFAD170477047002046
:102D400001E001C1121F002AFBD17047F0B51FB48A
:102D500086B00998089A030D0021024314D0514807
:102D6000514A1818504305141198012810981AD088
:102D7000281A401C00264D4F4D49009601910490A1
:102D8000002812DA444211E01198012449A30128D5
:102D900001D11098C1430698119A84600360C26003
:102DA00041600BB0F0BD4042E4E70446210500203D
:102DB0003F4A001C51410391029012E0E00707D006
:102DC00032463B4601990098FDF712FD01910090B3
:102DD00032463B4610461946FDF70AFD06460F46A9
:102DE0006410002CEAD10498039B0028029A0999E8
:102DF000089806DAFDF7FCFC019B009AFDF7F8FC49
:102E000005E0FDF79FFA019B009AFDF79BFA044647
:102E10000E460022284BFDF773FD03D80020C04367
:102E2000014607E00022254B20463146FDF72EFCE7
:102E3000FDF746FD102409E0002C0ADB0A220023DE
:102E4000FDF754FB079B30321A55641E02460A43B5
:102E5000F2D11122641C079B121B1C19119B012B20
:102E600003D0012308430ED10AE0084304D0112007
:102E700010900020119077E71098151A6D1E0BE046
:102E80001098824202DD00236D1C03E0824201DAC9
:102E900000236D1E002BEED0069811998260C16050
:102EA00030C07EE701FCFFFF104D00000000144021
:102EB0000000F03F300000000000F0430000E03F61
:102EC000FFB597B00646002518E2252877D10024E3
:102ED0002746FD49049400E00443761C3278012023
:102EE000203A90400842F7D130782A280ED00222AA
:102EF000307801463039092916D804990A235943F4
:102F0000303940181443761C0490F1E7189802C831
:102F100004911890002904DA012040030443484238
:102F2000049002200443761C30782E2814D104200B
:102F300004437078761C2A2809D11898761C80C81A
:102F4000189009E00A214F43303FC719761C3078AA
:102F5000014630390929F5D930786C2810D006DCC3
:102F60004C281AD068280ED06A2817D104E074289B
:102F700013D07A2812D110E00120400504430CE060
:102F80000121090501E0032109050C437178814203
:102F900003D1012000052418761C761C307811908E
:102FA00066280BD013DC58287DD009DC00287BD0A4
:102FB0004528F6D04628F4D047281AD1A5E118E0D4
:102FC000632835D0642870D0652812D19DE170281F
:102FD0006CD008DC6728F1D069287BD06E280DD032
:102FE0006F2806D1BAE073282ED0752871D07828C2
:102FF00059D01A9A199990476D1C7EE16002400FD2
:10300000022809D003280DD00428189801680DD093
:103010000D60001D189070E11898EA1701680D60A6
:103020004A60F6E7189801680D80F2E70D70F0E746
:1030300018986A4601781172001D1890002050728D
:1030400002A80090012005E0189802C818900020FE
:103050000091C04361070DD5002101E00199491C91
:103060000191B94212DA8142F8DB009A515C0029E1
:10307000F4D10BE0002101E00199491C019181424A
:10308000FADB019A0099895C0029F5D1019904982D
:103090001A9B471A21463846199A00F097FA019967
:1030A000401945180BE04FE02CE113E04EE000988A
:1030B00000990078491C00911A9A19999047019833
:1030C000401E0190401CF2D1214638461A9B199AA5
:1030D00010E137E00A200021009001916002410FC9
:1030E000022907D0189A01CA1892C21794460329D8
:1030F00008D00AE01898C01DC108C90005C9189178
:10310000944607E000B2C2179446042902D140B2A7
:10311000C1178C4600226146944506DA0A46002112
:10312000404291418C462D2102E0210504D52B21FE
:103130006A461173012103E0E10701D02021F7E77E
:10314000029155E00A200AE0102008E010200090CB
:103150000021042004430191082703E008200021F6
:10316000019100906002410F022907D0189A01CA0C
:10317000189200229446032908D008E01898C01D30
:10318000C108C90005C91891944603E080B204291A
:1031900000D1C0B200210291210729D511997029CF
:1031A00006D0009A1021019B4A401A4305D00EE038
:1031B00040216A461173012108E06146014306D0AF
:1031C00030216A4611731199517302210291009ABC
:1031D0000821019B4A401A430AD16146014301D1AB
:1031E000610705D530216A46117301217F1E0291C6
:1031F0001199582904D035A10E910DA90D910DE01A
:1032000037A1F9E76146019B009AFDF76FF90E9B24
:103210008C469B5C0D9A521E0D92137061460143C1
:10322000F0D10D9805A9081A20300190600703D548
:1032300001200004844300E001270198874201DD5A
:10324000381A00E0002001990090411802980918EE
:103250000498401A0490E00306D421461A9B199A58
:10326000049800F0B3F94519002706E003A81A9A5C
:10327000C05D199990476D1C7F1C02988742F5DB51
:10328000E0030CD521461A9B199A049800F09EF988
:10329000451904E01A9A3020199990476D1C00993D
:1032A000481E00900029F5DC08E00D980D99007883
:1032B000491C0D911A9A199990476D1C0199481E45
:1032C00001900029F1DC63E109280100303132333B
:1032D0003435363738396162636465660000000052
:1032E000303132333435363738394142434445463C
:1032F0000000000000F05AF94519761C30780028CB
:1033000000D0E2E528461BB0F0BD600700D40627D8
:103310001898C01DC108C90048680A680831C30F61
:10332000DB071891190001D09CA108E0210501D507
:103330009BA104E0E10701D09AA100E09AA143001B
:1033400011985B08109165280CD006DC452809D03F
:1033500046281DD0472841D141E0662818D067286B
:103360003CD13CE00021112F01DB112000E0781C52
:103370000191009008A911A8FFF7E8FC13990591A5
:103380000021119A15927F1C12980197009150E02C
:103390000120C00703900120019008A9009711A8FF
:1033A000FFF7D4FC139A149905920022119B009206
:1033B00012981593059A0192002901D0104602E057
:1033C000791C40180190381A01D5019804E0404258
:1033D000401E0090781C0190C01B029043E0012F1A
:1033E00000DA01270021112F01DD112000E038460D
:1033F0000191009008A911A8FFF7A8FC1399059165
:10340000119A0021129815920091019721070CD46E
:103410000599B94201DB019900E00191012904DD20
:10342000159A491E515C302906D0B84201DA011DB7
:1034300005DA0121029115E00199491EEDE7002806
:1034400005DC0099411800910199091A03E0019ADD
:10345000411C914200DD01910099401A401C0290EC
:103460000120C0070390200706D4029901988142E9
:1034700002DB0020C043029000206946C87707AFF6
:10348000012103980337C907884224D002201190F4
:103490002B201290039800280CDA404203902D2034
:1034A000129007E00A210398FCF73EFE30317F1EA0
:1034B000039039701199481E11900029F2DC03988D
:1034C0000028EFD1791E129808703078202108402A
:1034D0004530BF1E387006A8C01BC01D0390109851
:1034E0000078002800D00120019941180298C017E7
:1034F0000918039809180498401A401E0490E00324
:1035000006D421461A9B199A049800F05FF84519D1
:1035100010980078002803D01A9A199990476D1CCA
:10352000E00324D521461A9B199A049800F04EF81E
:1035300045191CE00098002807DB0099059888428F
:1035400003DD1598405C199901E0199930201A9A09
:10355000904700986D1C401C00900298401E0290FD
:10356000002804D11A9A2E20199990476D1C0199B0
:10357000481E01900029DDDC05E038781A9A7F1C8E
:10358000199990476D1C0399481E03900029F4DC9B
:1035900021461A9B199A0498ACE600002D00000001
:1035A0002B0000002000000000000000F8B50446D9
:1035B00000251E461746880404D405E0394620201D
:1035C000B0476D1C641EF9D52846F8BDFFB504460A
:1035D000002581B01E46C80301D5302700E0202712
:1035E000880404D505E038460399B0476D1C641E75
:1035F000F9D5284605B0F0BD70B504460D46E1B2D8
:103600000548FFF7B4FA00BF80210348FFF7CAF965
:103610000028F9D0204670BD001C0140FEF7AAF832
:103620000120FEF745FAFEF7DFFA0446012C34D1FB
:10363000FDF7FEFB0120FDF70DFC0020FEF786FAEA
:10364000A1048810FEF770FA0120FEF759FA00BFB6
:103650001920FEF7F1F90028FAD00220FEF784FACB
:1036600000BFFEF70DFA0828FBD10020FEF710FA84
:103670000020FEF733FA01200007FEF783FA01204D
:103680004007FEF77FFA03200007FEF77BFA1020C1
:10369000FEF716FA8020FEF799FAFEF787FDFFF78E
:1036A0004FFAFDF7E5FBFFF7A5F8FDF760FF642093
:1036B000FDF77EFBFF2101310920C006FDF776FDF5
:1036C0006420FDF775FBFF2101310920C006FDF7DD
:1036D0006FFDFFF751FAFEF79FFE1348FDF748FB19
:1036E000FEF7B2FC11490620FDF706FF1BE010486B
:1036F0000078012815D10F480078002804D001284F
:1037000005D0022809D105E0FDF7E8FF05E0FDF747
:1037100083FA02E0FDF70EFB00BF00BF0020044962
:103720000870FDF705FFE2E7B80B0000FF0F00008F
:103730002600002025000020424DE20000017142D9
:103740004DE100000170424DE100010171424DE484
:1037500000000173424DE400010174FF0186000086
:1037600000000079FF019900000007D08FFF019948
:103770000000001388CBFF019900000027102FFFE5
:103780000186000000000079FF01780400000000BD
:1037900083FF0186030000000084FF018600000013
:1037A000000079FF0178410000000046FF017840E9
:1037B000000000004700000041542B4C5253454E7E
:1037C000443D3130312C302C31382C3C253032788E
:1037D00025303278253032782530327825303278ED
:1037E00025303278253032782530327825303278DD
:1037F00025303278253032782530327825303278CD
:1038000025303278253032782530327825303278BC
:10381000253032780D0A00003838000800000020FA
:103820005C0000002E2D0008943800085C00002089
:10383000BC0600003E2D0008006CDC020000000009
:103840000000000001020304060708090000000050
:103850000102030401020304060708090201000033
:103860000000000000000000000000000000000058
:103870000000000000000000000000000000000048
:103880000000000000000000000000000000000038
:043890000000000034
:04000005080000BD32
:00000001FF
